:020000040000FA
:06000000D4EF07F012002E
:0600080004EF08F01200F5
:060018000CEF08F01200DD
:020020000000DE
:0E002200F00E8B1694160201A36BA769A86955
:10003000A969A66B010EAA6F1200D9CFE6FFE1CF26
:10004000D9FFE6520201A3511FE1020108BF1BD0F4
:10005000400EE66EA50EE66E000EE66E09EC06F0AA
:10006000E552E552E5520201010EA36FDF6A400E30
:10007000DF5C09E2DF50EA6A600FE96E000EEA22F7
:10008000EF6ADF2AF4D796D10001A551080A01E1F1
:1000900080D10F0A01E123D1010A01E118D1030A3D
:1000A00001E1B4D0010A6AE0070A5DE0010A01E05B
:1000B00081D10001020E606F00013A0E616F0001F4
:1000C000010E626F0001010E636F0001646B100E80
:1000D000656F666B676B0001686B300E696F6A6BEA
:1000E0006B6B0001030E6C6F00016D6B6E6B300E5D
:1000F0006F6F706B00010E0E716F726B736B746BB0
:100100000001010E756F0001766B776B200E786F22
:10011000796B0001080E7A6F7B6B7C6B7D6B000145
:100120007E690001020E7E6F00017F6B806BF00E16
:10013000816F826B0001836B010E846F856B866B10
:100140000001876902010CBF0DD0400EE66E600E03
:10015000E66E000EE66ED9EC05F0E552E552E5528A
:100160000201A36B27D10201010EAA6F0001A65163
:1001700002E10201AA6B0201A36B1CD1400E020135
:10018000A46FA56B0201000EA45D010EA5591FE22C
:100190000400A4C200F0A5C201F0026A060E1F0B03
:1001A00000C0F6FF01C0F7FF02C0F8FF06E0D890DC
:1001B000F636F736F836E806FAE1940EA66EA3D9BD
:1001C00063EC06F00201A42B000EA523DBD7DF6A47
:1001D000DF50A96EA868040EA66E63EC06F093D9F2
:1001E000DF50DF2A006E016A026AFF0E005C000E1B
:1001F0000158000E0258ECE3F66AF76A200EF86E1A
:10020000940EA66E80D90201A36BD4D0300E0001EB
:10021000A85D07E10201AA5101E132D90201A36BF5
:10022000C9D0F00E0001A85D04E14DD90201A36B15
:10023000C1D0E8680201A71905E1E868A81902E140
:10024000E868A91906E1A6C0A7F2A7C0A8F2A8C04D
:10025000A9F2A70EE96E020EEA6EEE500001A61991
:1002600008E1EE500001A71904E1EE500001A819C1
:1002700000E12AE1DF6A0001AA51DF5C25E23A0EC3
:100280000001D880AA55DF24EA6AAB0FE96E000EA0
:10029000EA22EF50E66E0201A651EA6AAB0FE96E60
:1002A000020EEA22E552E750EF6E0201A62B020190
:1002B000A72B000EA823000EA923100E0201A65D95
:1002C00001E17DD8DF2AD7D70201A36B73D077D89D
:1002D0000201A769A869A9690201A36B6BD000019B
:1002E000070E606FA6C061F0A7C062F0A8C063F0FF
:1002F000A9C064F0AAC065F0A6C0F6FFA7C0F7FFCA
:10030000A8C0F8FFDF6A0001AA51DF5C31E2F00EFD
:100310000001A85D13E1DF500001A625A96EA66AC1
:10032000A6803A0E0001D880AA55DF24EA6A660F3B
:10033000E96E000EEA22A8CFEFFF18D00900300EB8
:10034000F85C08E1050EF65C01E1F568080EF65C64
:1003500001E1F5683A0E0001D880AA55DF24EA6A67
:10036000660FE96E000EEA22F5CFEFFFDF2ACBD74A
:1003700002010CBF0DD0400EE66E600EE66E000E60
:10038000E66ED9EC05F0E552E552E5520201A36BA9
:1003900011D06492646ADF6AFF0EDF5C09E2E868EC
:1003A000E85004E0E80600D000D0FAD7DF2AF4D7FE
:1003B000FF0000D0E552E552E7CFD9FF120000015F
:1003C000A16BA6C200F0016A026A00500201A75D9B
:1003D000F66E01500201A859F76E02500201A959A8
:1003E000F86E0F0EF6140001A26FF00EF616000163
:1003F000A06B100E0001A05D1FE20001A25115E1EB
:100400000201A6510FE00001A151EA6AAB0FE96EAB
:10041000020EEA22EF50F56E0D000001A12B020141
:10042000A60702D0F5680D0004D0F5680D000001A4
:10043000A2070001A02BDDD70A00A40EA66E63D888
:100440000001A06B0201A6510001A05D18E20001AD
:10045000A1510001A025EA6AAB0FE96E020EEA2263
:10046000EF50E66E0001A051EA6AAB0FE96E020E92
:10047000EA22E552E750EF6E0001A02BE3D712000D
:10048000A6C0F6FFA7C0F7FFA8C0F8FF0001A36B46
:100490000001AA510001A35D15E23A0E0001D880C7
:1004A000AA550001A325EA6AAB0FE96E000EEA2205
:1004B000EF50F56E0C00C40EA66E25D809000001A1
:1004C000A32BE6D712000001A46B0001AA51000182
:1004D000A45D18E20001A6510001A425A96E3A0E00
:1004E0000001D880AA550001A425EA6AAB0FE96E85
:1004F000000EEA22EF50A86E040EA66E04D800018A
:10050000A42BE3D71200F29E550EA76EAA0EA76E7B
:0A051000A682A6B2FED7A694120040
:06051A007DD9E65263509A
:1005200032E16296020100513C0BE842E8420D08BC
:1005300028E1180E021923E1020E031920E1100E22
:10054000026F020E036FDF6ADF50006E016A080E51
:10055000005C000E015813E2DF50EA6A180FE96EE2
:10056000020EEA22EF50E66EDF50EA6A100FE96EE3
:10057000020EEA22E552E750EF6EDF2AE5D70ED8E9
:100580000AD03FD808D0040E635C03E1629650D8CD
:1005900002D0000E01D0010EE55242D13CD9E65204
:1005A000020104BF046B0201FD6BF56BF66BFB6B84
:1005B000FC6B1CEC04F0DF6ADF50006E016A010E78
:1005C000005C000E01581AE20201F65117E1F76AC9
:1005D000DF34FE0BF736F66EA00EF6260E0EF7226F
:1005E0000900F5CF00F00800F5CF01F004D001C0FC
:1005F000FAFF0050F96EFBDFDF2ADED7B7D8E552ED
:100600000FD1020E0201F55D0EE184D80201180E31
:10061000026F020E036F080E016F00BD02D0C80EFC
:1006200005D0880E03D0DBD8E7D88C0E006F1200FF
:10063000040E0001E55D0CE112C25CFF0F015C518C
:10064000000803E20001050E02D00001030EE56F71
:100650000201F50510E111D8020E0201FD5D03E172
:100660000201840E06D0020104BD02D0C80E01D0E2
:10067000880E046F1200EFEF03F0CDD8020EE126D2
:100680000201080EFB5D000EFC590DE2FBC2DEFF0D
:10069000FCC2DDFFFD5102E1010E03D0FD0506E1C4
:1006A000020EFD6F03D0080EDE6EDD6A02010493B8
:1006B0000491010EDB500413DFCF05F2000EDB5076
:1006C0000201FB5F010EDB50FC5B180EF96F020E9E
:1006D000FA6F0001E6A30CD097D815E0F7C2F6FF39
:1006E000F8C2F7FF0800F5507FD8F6E2DB06F4D732
:1006F0008BD809E0F7C2E9FFF8C2EAFFEF5074D8DF
:10070000F7E2DB06F5D7020EE15C02E2E16AE552B0
:10071000E16E86D080D8020EE126030E020100159C
:10072000E76E010EE7CFDBFF01C2DFFFDE50020103
:10073000FB27DD50FC23180EF76F020EF86F64D80C
:100740000EE0F7C2E9FFF8C2EAFFEF50F9C2E9FF95
:10075000FAC2EAFFEF6E68D8F2E2DB06F0D7020ECB
:10076000E15C02E2E16AE552E16E5AD0649802016E
:10077000F65105E141D8840E006F02011DD002013F
:1007800010AF1CD00201FB510201165D0201FC51A9
:100790000201175904E216C2FBF217C2FCF26DDF28
:1007A0000201010EF56F28D8800E006F0201180EAD
:1007B000066F020E076FC80E046F12000201020ED0
:1007C000F56F0201056BC80E046F0201080E016F80
:1007D000180E026F020E036FC80E006F12000201A6
:1007E000F56B0201046B1200F9C2E9FFFAC2EAFFDD
:1007F000EF6E020114EF04F00201080E016F100EFB
:10080000026F020E036F1200D9CFE9FFDACFEAFFC1
:10081000EE50ED101200D9CFE6FFE1CFD9FF120064
:10082000E552E7CFD9FF1200F92B000EFA23F72B80
:08083000F823DF06010E12009F
:0808380002011051600BE842BF
:10084000E842E842E842E842000901E012001151A2
:10085000070A40E00B0A3EE0070A33E0010A23E002
:100860000B0A1FE0020A1DE0030A19E0080A10E063
:10087000010A0CE00F0A08E0030A01E0120012D995
:100880000001040EE56F12006BEF04F0A2EF04F01C
:1008900009D90201E70EF76F000EF86F0CD0BDEF1B
:1008A00004F0EFEF04F002D90201F76FF86BE80EE5
:1008B000F727000EF8230001E6930201010EFB6FFB
:1008C0001200F4D8EA6AE80FE96E000EEA2212C2BA
:1008D000EFFF12001200800E0201105D32E1135191
:1008E000030A1FE0010A0AE0030A29E1DBD802013A
:1008F000E00EF76F0D0EF86F120E1ED0B2D8960EE6
:10090000F6260E0EC0D8020E0201F76AF725F66E23
:10091000F851F7220900F5CFFBF20A00F5CFFCF2FF
:100920000ED09FD89A0EF6260E0EADD8F7C2F6FF5F
:10093000F8C2F7FF0800F5500201FB6FFC6B0001E5
:10094000E6831200AFD8070EE66E540EE66E0F0E69
:10095000A2D8010EE66EE80EE66E000E9CD812C21A
:10096000E7F00201125104E10001050EE56F1200EB
:100970000001060EE56FC3EF05F00201186B196B5D
:10098000020110511F0B020A0FE0030A0BE0010ADB
:1009900018E188D8020118810001E6A112D00201F5
:1009A00018830FD07FD80DD050D801E0010E62D847
:1009B000F9C2E9FFEA6EEF50040B03E00201010EF9
:1009C000186F0201F6050AE10201180EF76F020E18
:1009D000F86F0001E6930201020EFB6F12000201A4
:1009E00012050EE110511F0B00090AE15BD8030E3E
:1009F0000201115D03E10001E68102D00001E691F0
:100A00000201125121E110511F0B02081DE1145186
:100A10000F0B000919E019D801E0010E2BD8030EC5
:100A20000201115D02E1840E03D014AF07D0400E25
:100A3000F9C2E9FFFAC2EAFFEF6E1200880EF9C2AE
:100A4000E9FFFAC2EAFFEF6E120030D80F0B080D73
:100A5000F350016A000F006E020E01221451800B48
:100A6000120020D802011251F66EF76AD890F636BD
:100A7000F7361200040DF35002010024F96F000E46
:100A80000120FA6F1200F7220900F5CFF7F20A00F1
:100A9000F5CFF8F21200E66EDBEC06F0E552E55217
:100AA000E55212000201010EF66F1200FBDF020197
:040AB00014511200CB
:0C0AB400020110511F0B010801E01200AC
:100AC000145101E01200060E115D24E11351230AB6
:100AD0001FE0010A0DE0030A1BE1DCD80001E70575
:100AE00005E10201040EF76F0E0EF86F090E0DD02E
:100AF000D1D80001E70505E10201790EF76F0E0E6E
:100B0000F86F0001E70504E11D0E0201FB6FFC6BAD
:100B10000001E68302011051600BE842E842E8421E
:100B2000E842E842010801E0120011510B0A25E0F9
:100B3000080A17E0090A11E0080A09E00B0A05E0B3
:100B4000080A01E01200C1EF05F0C2EF05F0A2D8DB
:100B50000201E90EF76F000E09D09CD813C2E9F02C
:100B6000120098D80201EA0EF76F000EF86F00012C
:100B7000E6930201010EFB6F12008CD812C2EAF05C
:100B80001200120012000001EB6B0F011E0E546FD9
:100B90000201400E096F200E0A6F020E0B6F880EC5
:100BA000086F0201600E0E6F020E0F6F400E0C6F89
:100BB0001200D9CFE6FFE1CFD9FFE652FC0EDB50A1
:100BC000400805E2400EF36EFC0EF3CFDBFFDF6A58
:100BD000FC0EDB50DF5C0FE2DF5050D8EF50E66ECA
:100BE000DF50EA6A600FE96E020EEA22E552E75032
:100BF000EF6EDF2AEDD7FC0EDBCF0DF2400E0201C7
:100C00000C170C7D880E0C13E552E552E7CFD9FF87
:100C10001200D9CFE6FFE1CFD9FF0001EB6B020153
:100C200008BF26D0FC0EDBCF00F00951D88000545D
:100C300003E2FC0E09C2DBFF0001EB6BFC0EDB5094
:100C4000EB5D0FE2EB51EA6A200FE96E020EEA2239
:100C5000EF50E66EEB5112D8E552E750EF6EEB2BFA
:100C6000EDD70201400E096F0817087D880E0813A2
:100C70000001EB51E552E7CFD9FF1200E76EFD0E00
:100C8000DBCFE9FFFE0EDBCFEAFFE750E926000EDF
:0C0C9000EA2212000201020EF66F1200B0
:040C9C0064A60CD866
:100CA0000001E50508E164BA06D0626A606A608006
:100CB0006088020EE56F1200646A606A6486000153
:100CC000010EE56F12000001E55101E1120062B46E
:100CD00025D864B2120062B03AD862B817D862BAA6
:100CE00024D8030E0001E55D01E212000201FE6B53
:100CF000040EFE5D0AE262A608D08DEC02F0000947
:100D000001E162960201FE2BF3D712006084629823
:100D10006482A194A0840300A09412006492609461
:100D200062A402D06294FCD712000F0153A10DD02F
:100D3000800E0201005D07E1840E0201045D03E103
:100D400002018C0E006F0F015391629A12000F0185
:100D50005F6B626A0F019F0E5B6F7B0E606E0F010F
:100D60005C6B070EE66E540EE66E0F0EE66E23D831
:100D7000E552E552E5520F01160E536F62A605D0FB
:100D8000629600D000D00000F9D76498EFEC03F031
:100D90000201080E016F0201100E026F020E036FB6
:100DA00002018C0E006F0001E6910001E76B00016B
:100DB000030EE56F1200D9CFE6FFE1CFD9FFFD0E9C
:100DC000DBCFE9FFFE0EDBCFEAFFFC0EDB5004E0D9
:100DD000EE6AFC0EDB06F9D7E552E7CFD9FF120029
:100DE0001201000200000008D8043C0002000102C9
:100DF000000109022900010100C0320904000002BB
:100E000003000000092111010001221D00070581D6
:100E100003400001070501034000010403090434F5
:100E2000034D006900630072006F00630068006991
:100E3000007000200054006500630068006E006FC1
:100E4000006C006F0067007900200049006E0063AD
:100E5000002E00260348004900440020005500539E
:100E6000004200200042006F006F0074006C006FB1
:100E70000061006400650072000600FF0901A10125
:100E800019012940150026FF0075089540810019B9
:100E90000129409100C0F20DF20D1B0E1F0E530EE2
:020EA000B40A92
:0E0EA200200EF66E000EF76E000EF86E0201C6
:100EB0000900F550F06F0900F550F16F03E1F0679C
:100EC00001D03DD00900F550EB6F0900F550EC6FF3
:100ED0000900F550ED6F09000900F550E96E0900B1
:100EE000F550EA6E090009000900F550EE6F09009F
:100EF000F550EF6F09000900F6CFF2F2F7CFF3F2E9
:100F0000F8CFF4F2EBC2F6FFECC2F7FFEDC2F8FF48
:100F10000201EE5302E1EF5307E00900F550EE6ED7
:100F2000EE07F8E2EF07F9D7F2C2F6FFF3C2F7FFD8
:100F3000F4C2F8FF0201F007000EF15BBFD7120008
:100F40000F0EC16E82A804D0070EC16E00EF08F02C
:100F50000DD8040015D8060E0001E55D05E16450CA
:100F6000020B02E11DEC00F0F4D71200140E616ECA
:100F70000001E56B0001E66B0001E76B11EF00F08B
:080F80004EEC06F063EF06F0F1
:080F8800000EF36E00EE00F014
:100F9000030E01D81200EA6002D0EE6AFCD7F350CB
:080FA000E9601200EE6AFCD7C3
:080FA80011EE00F021EE00F053
:100FB000F86A049C51EC07F0E2EC07F0A0EC07F0B3
:040FC000FBD7120049
:020FC400120019
:020000040030CA
:0100000000FF
:0100010032CC
:0100020001FC
:010003001EDE
:0100050000FA
:0100060001F8
:0100080003F4
:01000900C036
:01000A0003F2
:01000B00E014
:01000C0003F0
:01000D0040B2
:00000001FF
